:100000008829AE0006300428A7002F082D02031D02
:100010000B282E082C02043003180130031902307B
:100020002705031D013083298030A100FE30C22046
:100030000130C2207530AD0030303D29A101A1173B
:10004000B500B508031D2628030127280130B50295
:100050000310A20CA20CA20CC0302205403EB50732
:10006000FE30C2203508C228A101A117B500FE301C
:10007000C2203508C228A501B000B101A011250891
:100080000319A0150530A4002730AF00103054200C
:100090000330AF00E8305420AF0164305420AF018A
:1000A0000A30542030085B28AE003108AD0030081B
:1000B000AC0051212C08AC00A4030319A0112508A1
:1000C00003196528240203186C282C08031DA011AD
:1000D000A0196C28303EC2280800A4002508031986
:1000E00083292408C220A5036E28B30085100510BB
:1000F0008316851005100F30860583123308A0186B
:100100009F283E30AD0080303D213330B200B32017
:100110001330AD0088303D21B32064303C21B32042
:1001200064303C212230B200B32028309E200C30B5
:100130009E2006309E20A01433089F282014B20071
:10014000201CAD280510033C031CB228B22005304A
:10015000AD00DC303D21031408002014FE3C0319DF
:10016000C0280514201C201085140F308605320885
:10017000F03986048510B20E2018B32832303C21A5
:1001800033088329A11B7528AE00083027190130D8
:10019000AF00AE0C220884002608CE28CF28FF3AF4
:1001A0008005841780052608031880043C303C2114
:1001B00026088004AF0BC9280314832908302719A7
:1001C0000130AF00AE01220884002608FF3A800506
:1001D000841780052608800407303C2126088413F4
:1001E0000005FF3E271DAE0C2719AE0D32303C2115
:1001F000AF0BE5282E0803148329A71C83290329A4
:10020000A700271C8329220884002608FF3A8005BE
:10021000841780050130AD00F4303D2126088004AC
:100220000130AD00F4303D2983169B0083161C1469
:100230001A089B0A832983169A001C1555309D00C5
:10024000AA309D009C149C1823291C119B0A832909
:1002500083178001840AFF3E031D29298329AF01EA
:10026000AE00FF30AE07031CAF07031C8329033029
:10027000AD00E5303D213129AD01F63EAC00AD09C0
:10028000031C4829FE300000AC0703184329AC07C3
:100290000000AD0F422900002C184E292C185029BF
:1002A0000800B101B0011030B2002D0DB00DB10D3C
:1002B0002E08B0022F08031C2F0FB1020318672964
:1002C0002E08B0072F0803182F0FB1070310AC0D2D
:1002D000AD0DB20B55292C0883291030B700AD01A4
:1002E000AC01B30CB20C031C7B292E08AC072F0801
:1002F00003182F0FAD07AD0CAC0CB10CB00CB70B45
:100300007129300883298313831203130000080026
:10031000A00107309F00F73083168500FF3086006C
:1003200081138312850186012030840060308A01A8
:100330002921A030840050308A01292120308400F6
:1003400050308A0128210130AF002C308A01302141
:10035000FA308A011421ED00FB308A011421831642
:10036000A000FC3083128A011421A8008A01162102
:10037000A9002908C0002808BF00FE308A01142106
:10038000A8008A011621A9002908C2002808C10076
:10039000FF30FD000F3006058316A3000F30230247
:1003A0008A1183120318E429ED0AFA3083169B00A0
:1003B00083126D088A011B218A116D18E1298316A9
:1003C000A00183128A11422A8A01142049308A012D
:1003D00075206E308A01752066308A0175206F3075
:1003E0008A01752072308A0175206D308A0175206E
:1003F00061308A01752074308A01752069308A0164
:10040000752065308A01752020308A0175206F3093
:100410008A01752070308A0175208030A100C030BB
:100420008A01342077308A0175208A0175208A017B
:1004300075202E308A01752070308A017520693050
:100440008A01752063308A01752062308A01752027
:1004500061308A01752073308A01752069308A0104
:10046000752063308A0175202E308A0175206E3028
:100470008A0175206C308A0175200B30AF00B830CE
:100480008A0130218A01142042308A0175206530AA
:100490008A01752074308A01752061308A017520C7
:1004A00020308A01752031308A0175208030A1000A
:1004B000C0308A01342057308A01752065308A01A6
:1004C00075206B308A01752065308A0175206E3089
:1004D0008A0175203A308A017520A50103016D1843
:1004E0000130013EB000B101B10D8A013E200B3058
:1004F000AF00B8308A013021FE308A0175204030CB
:100500008A01752003018A0175200C308A0175204B
:100510000C308A0175200C308A0175200C308A015C
:1005200075200F308A0175200F308A017520030174
:100530008A01752003018A0175201B308A0175200C
:100540001B308A0175201F308A0175201F308A01F7
:1005500075201B308A0175201B308A01752003012C
:100560008A01752004308A0175200C308A017520BB
:1005700004308A01752004308A01752004308A0114
:10058000752003018A01752003018A01752003018A
:100590008A0175200C308A01752012308A0175207D
:1005A00004308A01752008308A0175201E308A01C6
:1005B000752003018A01752003018A01752003015A
:1005C0008A01752003018A01752003018A017520C3
:1005D00003018A01752006308A01752006308A01E0
:1005E000752003018A01752003018A01752003012A
:1005F0008A0175201F308A01752019308A01752003
:1006000017308A01752017308A01752017308A014A
:10061000752019308A0175201F308A017520030169
:100620008A0175208A01142053308A0175206930AF
:100630008A01752067308A0175206E308A01752025
:1006400061308A0175208A0175206C308A0175201D
:1006500020308A0175207A308A0175206F308A0136
:10066000752065308A0175206B308A0175206530F0
:100670008A0175206E308A0175203D158A158A28F9
:10068000F1015E03A8008316A301831283162308D9
:10069000831228028A11031C682B8A118C238A1169
:1006A000BD1E622B7108AC00831623088312A200C2
:1006B000AC01A20A0314AC0DA2038A11031D5B2B2B
:1006C0002C08F1048316A30A8A118312031D452BFB
:1006D000B9017108B800B90CB80CB90CB80CB90C58
:1006E000B80CB90CB80C0F30B9053908B30038088C
:1006F000B200AF010A30AE008A016D21B8003108A6
:10070000B900BB017108BA000F30BA050030BB0553
:1007100038083A07F10008008A113E1C912B8A150F
:100720008A28D401D3018A11051AAD2B01308A0120
:100730002F21D30A0319D40A0B3054028A11031C47
:10074000AB2B8A11031DA92BB93053028A11031C4C
:10075000AB2B8A15EB2A8A01932BDC01DB015C08A9
:100760008A11031DC22B9B305B028A110318C22B16
:10077000DB0A0319DC0A01308A012F218A1158276C
:100780008A01AF2B051ABD16051EBD128A113D1D2B
:10079000DA2B0310750CE2000310E20C8030A1008C
:1007A0000230A20062088A012020FF308A017520F1
:1007B0008A11E52B0301BD1B013EBD1A013A031945
:1007C000BD13031DBD178A110724F50ADC01DB01E7
:1007D00002305C02BC3003195B028A110318FA2B49
:1007E000DB0A0319DC0A01308A012F218A115827FC
:1007F0008A01E82B01306A028A11031D012C8A113B
:10080000EA24EA088A110319062CEA030800C73013
:100810008A013420A10104308A0175208A113E1E0C
:10082000162C01308A0175208A11192C03018A01C6
:100830007520A5308A01752008008030A100C030E5
:100840008A01342063088A013B2020308A01752008
:1008500001306B028A11031D382C6A308A01752021
:1008600061308A0175206E308A0175208A11E62C6C
:1008700002306B028A11031D482C66308A017520F4
:1008800065308A01752062308A0175208A11E62C54
:1008900003306B028A11031D582C6D308A017520BC
:1008A00072308A01752074308A0175208A11E62C15
:1008B00004306B028A11031D682C61308A01752097
:1008C00070308A01752072308A0175208A11E62CF9
:1008D00005306B028A11031D782C6D308A0175205A
:1008E00065308A01752069308A0175208A11E62CED
:1008F00006306B028A11031D882C6A308A0175202C
:1009000075308A0175206E308A0175208A11E62CB7
:1009100007306B028A11031D982C6A308A017520FA
:1009200075308A0175206C308A0175208A11E62C99
:1009300008306B028A11031DA82C61308A017520D2
:1009400075308A01752067308A0175208A11E62C7E
:1009500009306B028A11031DB82C73308A0175208F
:1009600065308A01752070308A0175208A11E62C65
:100970000A306B028A11031DC82C6F308A01752062
:100980006B308A01752074308A0175208A11E62C3B
:100990000B306B028A11031DD82C6E308A01752032
:1009A0006F308A01752076308A0175208A11E62C15
:1009B0000C306B028A11031DE62C64308A0175200D
:1009C00065308A01752063308A01752020308A01E4
:1009D000752008008A113D1DEE2C0800CA308A01DE
:1009E0003420A10103305602E830031955028A1160
:1009F0000318FD2C20308A0175208A113D1A032D21
:100A000020308A0175208030A10003013D1A013099
:100A1000A5002D308A016D20A5015608AD005508AE
:100A2000AC00AF016430AE008A015121B0002D0846
:100A3000B1008A013E202E308A0175200130A500C8
:100A40005608AD005508AC00AF010A30AE008A016F
:100A50005121B0002D08B1008A013E20DF308A010B
:100A6000752008008B308A013420A10172088A1198
:100A7000031D512D0A307A028A110318422D2030AD
:100A80008A0175208030A1007A088A013B203A3023
:100A90008A0175200230A5006E088A013C208A1167
:100AA000602D8030A1000230A50072088A013C2030
:100AB00075308A0175208A01752072308A0175208F
:100AC00008008030A10080308A0134200A30A5005F
:100AD00020308A016D2080308A013420A10101304C
:100AE000831622028A118312031D8C2D4D308A0138
:100AF000752061308A0175208A0175206E308A0167
:100B0000752064308A01752061308A017520673054
:100B10008A0175208A11472E0230831622028A111B
:100B20008312031DAA2D44308A01752069308A0181
:100B300075206E308A01752073308A01752064300B
:100B40008A01752061308A01752067308A0175201D
:100B50008A11472E0330831622028A118312031D45
:100B6000CB2D57308A0175206F308A017520653092
:100B70008A0175206E308A01752073308A017520D4
:100B800064308A01752061308A01752067308A01DE
:100B900075208A11472E0430831622028A1183128F
:100BA000031DEF2D44308A0175206F308A017520B6
:100BB0006E308A01752064308A01752065308A01A3
:100BC000752072308A01752064308A017520613089
:100BD0008A01752067308A0175208A11472E0530F9
:100BE000831622028A118312031D0D2E56308A01AC
:100BF000752072308A01752069308A0175206A304B
:100C00008A01752064308A01752061308A0175205F
:100C100067308A0175208A11472E0630831622021A
:100C20008A118312031D2E2E5A308A0175206130DD
:100C30008A01752074308A01752065308A0175201B
:100C400072308A01752064308A01752061308A0112
:100C5000752067308A0175208A11472E0730831668
:100C600022028A118312031D472E5A308A017520F1
:100C70006F308A0175206E308A01752064308A01D8
:100C8000752061308A01752067308A0175208A11CC
:100C90006D1C522E02308316201B013E8312B000C1
:100CA0008A01752008000530A2000430A60001303A
:100CB000A7008A010021CC308A01C42044308A0177
:100CC000C42008000530A2000430A6000130A700AF
:100CD0008A010021CC308A01C420BE308A01C420A0
:100CE0000530A2000430A6000230A7008A01DE20F1
:100CF000D5008A01DE20D6008A01DE208316A300FB
:100D000083128A01DE208316A30083128A01DE206B
:100D10008316A30083128A01DE208316A3008312A8
:100D20008A01DE20F4008A01DE20F7008A01FD201E
:100D30003D12013056028A11031C9F2E3D16B90147
:100D40007708B8007408B802031CB9033908B30067
:100D50003808B200AF016430AE008A016D21B800DE
:100D60003108B9003908AD003808AC00AF01770888
:100D7000AE008A015121F8005608B3005508B200B0
:100D8000AF010530AE008A016D21D5003108D600D3
:100D90008A113D1EDD2E5508FA3CD5005608031C6D
:100DA000013EFF3CD6007808643CF80033307802FE
:100DB0008A110318DD2E6430F8075608B90055086B
:100DC000B8002630B80702300318013EB9073908C9
:100DD000AD003808AC00AF010A30AE008A015121E5
:100DE000B8002D08B9003908B3003808B200AF01C7
:100DF0006430AE008A016D21B8003108B90078086E
:100E0000B8070318B90A7C303802D5001530031C26
:100E1000013E3902D6003F303E1A023E84000008EF
:100E2000A800840A0008A9002908B9002808B80009
:100E30003908B3003808B200AF010A30AE008A01A9
:100E40006D21B8003108B900BB010230BA000310AF
:100E5000BB0CBA0C3A08B8023B08031C013EB902AD
:100E6000030185190130BB01BA000310BA0DBB0D97
:100E700038083A07A80039080318013E3B07A900C3
:100E80005608AD005508AC002908AF0028088A01B3
:100E90000120BC0003013D1A01303C048A110319F2
:100EA000542F85158A11552F85118A01EA240800CF
:100EB0008A113D1D5C2F08005A0859048A15031D2C
:100EC00085280F300605F9000F3079028A150318BE
:100ED0007F283E14CB308A013420A10107307902EB
:100EE0008A11031D7C2F67088A11031D792F8A152B
:100EF000722BE7038A1536280A3079028A11031DFE
:100F0000A22F3F08A8004008A90029088A11031D44
:100F10008E2F333028028A11031C9F2F3F08AA000E
:100F20004008AB002B08A90005302A02A800031CCA
:100F3000A9032908C0002808BF00BD15BD14BE12B2
:100F40008A1536280B3079028A11031DC72F4108F4
:100F5000A8004208A90029088A11031DB42F4730B0
:100F600028028A11031CC42F4108AA004208AB00C2
:100F70002B08A90005302A02A800031CA903290890
:100F8000C2002808C100BD15BE168A1536280C30CF
:100F900079028A11031DED2F3F08A8004008A9001F
:100FA00029088A11031DEA2FB43028028A11031878
:100FB000EA2F3F08AA004008AB0005302A07A80026
:100FC0002B080318013EA9002908C0002808BF000B
:100FD000BD15BD14BE128A1536280D3079028A154A
:100FE000031D11284108A8004208A9000130290268
:100FF0004030031928028A1503180E284108AA0058
:101000004208AB0005302A07A8002B080318013E50
:10101000A9002908C2002808C100BD15BE168A15FE
:1010200036280E3079028A15031D36288A153E1996
:101030002E283E173E1E3E1383103E1E8314831837
:101040003E16831C3E128A15851A27283E123E152D
:10105000BE163E1EBE12F2018A1536286330720299
:101060008A1503183428F20A6E08F3000830790252
:101070008A15031C66288030A1000230A5003F308D
:10108000BE1A023E84000008A800840A0008A900D5
:101090002908AD002808AC00AF010A30AE008A0173
:1010A0005121B0002D08B1008A013E202E308A0166
:1010B00075200130A5003F30BE1A023E84000008B2
:1010C000B000840A0008B1008A013E200530EA0021
:1010D0008A15BD1C7228F2013E163E1F3E12BE1636
:1010E0003E1EBE128A153D187B288A01322501302A
:1010F000DA00F430D9008A0107248A158328BD104C
:101100000430E7003E118A158928D903590A0319CA
:10111000DA0308008A153D1C8F288A15EB2ADD01A9
:10112000F501BE108A15BE18592901306A028A15C8
:10113000031D9C288A01EA24EA088A150319A128BC
:10114000EA03D401D3018A15051EBF28D30A031967
:10115000D40A01308A012F213A3054028A15031C27
:10116000BB288A15031DB928993053028A15031C20
:10117000BB288A15EB2A8A0158278A15A3288A15C5
:10118000051AEF28D30A0319D40A01308A012F2146
:101190008A0158278A153D19DE28093054028A151C
:1011A000031CDC288A15031DDA28C53053028A1572
:1011B000031CDC288A15EB2A8A15ED283A305402E4
:1011C0008A15031CED288A15031DEB28993053025C
:1011D0008A15031CED288A15EB2A8A15BF28413091
:1011E0005D028A15031CF6288A15EB2ADD0A0330F6
:1011F00054028A15031C05298A15031D0429E930A8
:1012000053028A15031C0529BE148A153D1D572952
:101210005D0EB800B900F030B8050F30B9053908D7
:10122000AD003808AC00AF014130AE008A01512159
:10123000E2008030A10080308A01342053308A01DE
:10124000752069308A01752067308A0175206E30FB
:101250008A01752061308A0175208A0175206C3001
:101260008A01752020308A01752067308A01752037
:1012700065308A01752076308A0175206F308A01C9
:1012800075206E308A01752064308A0175206530C2
:101290008A0175206E308A0175208030A1000230ED
:1012A000A20062088A012020FF308A0175208A1579
:1012B00092288A153D1D98298A01142049308A01F7
:1012C00075206E308A01752069308A01752074306E
:1012D0008A01752069308A01752061308A01752084
:1012E0006C308A01752069308A01752073308A015B
:1012F000752065308A01752072308A01752065304D
:101300008A0175206E308A0175202E308A01752081
:101310008A0175208A0175208030A100C0308A01C1
:1013200034200E30A5005F308A016D208A15412AD5
:101330008A153E1CAF293B306E028A150318A3297B
:10134000EE0A8A15AD29EE0117307A028A150318C4
:10135000AC29FA0A8A15AD29FA018A15BB29803011
:10136000A1008A308A01342020308A0175206F085C
:10137000EE007B08FA0073086E028A15031DC5296A
:10138000F2088A150319C529F2038A013225720869
:101390008A15031D3D2A0730DF00B9017E08B80019
:1013A0000330AC000310B80DB90DAC038A15031D52
:1013B000D2290830B802031CB9035F08B807031824
:1013C000B90A0310B80DB90D831620088312380727
:1013D000E60066088A011421FC00660A8A011421CD
:1013E000F000B3017C08B200AF016430AE008A01A6
:1013F0006D21B8003108B90070083807A800390815
:101400000318013EA900B3017A08B200AF016430AD
:10141000AE008A016D21B8003108B9006E083807A6
:10142000AA0039080318013EAB0029082B028A15CF
:10143000031C362A8A15031D222A28082A028A1527
:10144000031C362A66087D028A150319342A6608A9
:10145000FD0001305F05B800B9013808013A0139D3
:1014600003193E12031D3E168A153B2A0130DF0286
:101470008A150318CD298A153F2AFF30FD008A01FD
:1014800062268A15BE1CE72ABD133E108316A301EF
:1014900083121530831623028A1583120318582AE3
:1014A0008A018C238316A30A8A158312031D482AF6
:1014B0008A0153260730DE008A0140237108EF00BD
:1014C0008A0162268A018C238A15BD1F682A3E1470
:1014D0000630DE008A0140237108FB008A018C235C
:1014E0008A15BD1F742A3E148A0153260630DE0079
:1014F0008A0140237108E4008A0162260330DE007D
:101500008A0140237108FF000530DE008A01402374
:101510007108EC000830DE008A0140237108E90000
:101520008A0153268A018C238A15BD1F982A3E14EE
:101530008A153E18D22A7F087E02A800A901031C42
:10154000A9032808063A29048A15031DB32A8A1517
:101550006D1CB32A70308316A006FB309B00200858
:1015600083128A011B216408E3007F08FE006C08D7
:10157000EB006908E8008A15BD1DD22ABD113F089D
:10158000E000FC3083169B00831260088A011B2157
:101590004108E000FE3083169B00831260088A0138
:1015A0001B213E148A153D1DDB2A8A153E18D92AB7
:1015B0003D118A0114207E088316A20083128A013D
:1015C00061258A011D248A0162268A15E92A8A1565
:1015D000EB2A8A158A283D143D118030A100803005
:1015E0008A01342047308A01752065308A017520D0
:1015F0008A0175206E308A01752020308A0175209D
:1016000044308A01752043308A01752046308A01B2
:10161000752020308A01752073308A017520693069
:101620008A01752067308A0175206E308A01752025
:1016300061308A0175208A0175206C308A0175201D
:101640003630A50020308A016D208A010724051A52
:101650003D17051E3D130301051A013E3D1B013CCC
:101660008A15031D6C2B0F300605A901A800290857
:101670008A15031D4D2B0F3028028A1503184D2B98
:10168000DA01D9018A0158270130E1000130AF00A9
:10169000F4308A0130218A15502B3E110430E700C6
:1016A000F60A643076028A15031D582BF601E10A0A
:1016B000023061028A15031D5F2B8A015326053013
:1016C00061028A15031C672B8A016226E1010A3038
:1016D0008A012F218A152B2B3D103D158A011420DC
:1016E0008A158A280130E50083162008A100A00190
:1016F0000B308312D800B830D700D7088A15031DE5
:10170000852BD8088A1503198B2F8A0114206508A8
:101710008316A20083128A01612596308316A300E6
:10172000193083128A012F218A158619B12B8A1547
:101730006D1CAF2B14308A012F218316A3032308BD
:101740008A158312031DAF2B70308316A106FB3060
:101750009B00210883128A011B218A15B12B8A154F
:10176000942B831623088A158312031DB92B8A151F
:101770008B2F0130D800F430D700D703570A031954
:10178000D8030A308A012F21580857048A15031DEF
:10179000CB2B8A15D52B093006058316A3000930FB
:1017A00023028A1583120318BD2B8A150618382FB9
:1017B000DF0108305F028A150318142CB90165088F
:1017C000B8000330AC000310B80DB90DAC038A1596
:1017D000031DE32B0830B802031CB9035F08B807E8
:1017E0000318B90A0310B80DB90D83162008831227
:1017F00038078316A300230883128A011421A80046
:101800005F084B3E8400280880008316230A831259
:101810008A011421A8005F08433E84002808800044
:10182000DF0A8A15031DD92BDF018A150618292C1A
:1018300006300605A901A80029088A15031D272CD2
:10184000063028028A150318272C8A15292C8A1598
:10185000152C8A15861D382F19308A012F210B303F
:10186000D800B830D7000F3006058316A3000E301D
:1018700023028A158312031D462CDF0A08305F02FB
:101880008A15031C442CDF018A15712E0D30831636
:1018900023028A158312031DBD2CBE155F08831613
:1018A000A30083120730831623028A1583120318BC
:1018B000682C8316A30A23084B3E84006330800003
:1018C0002308433E84000030800083128A15512C87
:1018D0005F084B3E84000008A800A80A5F084B3E42
:1018E0008400280880005F084B3E84000008A800A0
:1018F000183028028A15031CBB2CDF088A1503192F
:10190000B62C5F08433E84000008A8005F03433EF6
:1019100084000008AA002A082802013003180301E5
:10192000BC005F084B3E84000008A800633028021A
:1019300003190130031D03013C048A150319AA2C65
:101940005F03433E84000008A8005F08433E840014
:10195000280880005F034B3E84000008A8005F0851
:101960004B3E8400280880008A15BB2C5F084B3E44
:101970008400003080008A15712E0B3083162302FC
:101980008A158312031D4E2DBE155F088316A30012
:1019900083120730831623028A1583120318DA2C68
:1019A0008316A30A23084B3E840063308000831211
:1019B0008A15C82C5F084B3E84000008A8006330DD
:1019C00028028A15031D0A2D5F088A15031DF42CB1
:1019D0005F08433E8400003080005F084B3E840077
:1019E000003080008A15082D5F03433E8400000804
:1019F000A8005F08433E8400280880005F034B3E38
:101A000084000008A8005F084B3E8400280880007E
:101A10008A15172D5F08433E84000008AA00053090
:101A20002A07A8005F08433E8400280880005F085A
:101A3000433E84000008A8003C3028028A15031C9D
:101A40004C2DDF088A150319472D5F084B3E840093
:101A50000008A8005F034B3E84000008AA00280885
:101A60002A028A15031D402D5F03433E84000008AF
:101A7000A8005F08433E8400280880008A15452D91
:101A80005F08433E8400003080008A154C2D5F08BB
:101A9000433E8400003080008A15712E0C3083167E
:101AA00023028A158312031D902D023065028A15C8
:101AB000031C8E2DBE158030A100C0308A01342059
:101AC00005308A017520DF0108305F028A1503188E
:101AD0008D2D03105F0DB800B901B90D83162008D4
:101AE000831238078316A300230883128A01142166
:101AF000A8005F084B3E8400280880008316230A54
:101B000083128A011421A8005F08433E840028083C
:101B10008000DF0A8A15031D642DDF018A15712EEE
:101B20000A30831623028A158312031D192E0230F0
:101B300065028A15031C172E063065028A150318E4
:101B4000172E0330AF00E8308A013021053006053A
:101B50008316A30023088A158312031D172EBE11B6
:101B60008030A100C0308A01342005308A01752000
:101B7000DF0108305F028A150318162E03105F0D6F
:101B8000B800B901B90D83162008831238078316EF
:101B9000A30010308312E600413066028A15031854
:101BA000FC2D8316230883128A0114218316A400B6
:101BB00083126608831623079B00240883128A0178
:101BC0001B218316230A83128A0114218316A40081
:101BD00083126608831623078312B800B901B90D72
:101BE000380A83169B00240883128A011B211030B7
:101BF000E6078A15031CCC2D8316230883128A015D
:101C00001421A8005F084B3E84002808800083163A
:101C1000230A83128A011421A8005F08433E84002E
:101C200028088000DF0A8A15031DB92DDF018A15F7
:101C3000712E0930831623028A158312031D712E1B
:101C40000330AF00E8308A013021063006058316E4
:101C5000A30023088A158312031D712EBE158A0165
:101C600014208A0161258030A100C0308A0134200F
:101C700069308A01752073308A01752020308A010D
:101C8000752067308A01752065308A0175207730AC
:101C90008A01752069308A01752073308A017520A8
:101CA00074308A017520DF0108305F028A1503183D
:101CB000672E5F084B3E8400633080005F08433E20
:101CC000840000308000DF0A8A15031D542EDF01D6
:101CD0000F30AF00A0308A0130218A0114208A0120
:101CE00061258030A1008A308A01342062308A0167
:101CF00075206C308A0175206F308A0175206B3039
:101D00008A01752020308A017520A50102305F0705
:101D1000B800B901B90D0310390CB100380CB0008E
:101D20008A013E20C4308A013420A10101305F05C0
:101D3000A800A901290828048A15031DA92E4130ED
:101D40008A0175208A0175204E308A0175208A1516
:101D5000B22E55308A01752049308A0175205430E1
:101D60008A01752020308A0175206F308A01752024
:101D70006D308A01752020308A0175205F084B3E46
:101D800084000008A800633028028A15031DD72E9E
:101D90002D308A0175208A0175203A308A0175201C
:101DA0002D308A0175208A0175208A15EC2E80302D
:101DB000A1000230A5005F084B3E840000088A01A4
:101DC0003C203A308A0175200230A5005F08433E6E
:101DD000840000088A013C208316A3018312063088
:101DE0000605A901A80029088A15031D0B2F063036
:101DF00028028A1503180B2F8316A30A9730230293
:101E00008A158312031C062F8A150B2F02308A01B4
:101E10002F218A15EE2E0F300605A901A8002808EB
:101E20000E3A29048A15031D172F8A150B2FD70385
:101E3000570A0319D8030A308A012F21580857047A
:101E40008A15031D252F8A152F2F0F30060583169F
:101E5000A3000F3023028A1583120318172F580886
:101E600057048A15031D362F8A15382F8A15292CF9
:101E70008A15BE1D7A2FBE11DF0108305F028A1558
:101E800003187A2FB9016508B8000330AC000310BD
:101E9000B80DB90DAC038A15031D472F0830B802E1
:101EA000031CB9035F08B8070318B90A0310B80D7B
:101EB000B90D8316200883123807E6005F084B3EF1
:101EC00084000008E000660883169B008312600807
:101ED0008A011B215F08433E84000008E000660A77
:101EE00083169B00831260088A011B21DF0A8A1572
:101EF000031D3D2FE50A083065028A15031C892F52
:101F00000130E5008A156D1C882F70308316A006FD
:101F100083128A157D2B8A01142083162108A000C4
:101F200083127E088316A20083128A0161258A012A
:101F3000EA248A011D248030A1008A308A013420DD
:101F40002A308A0175208A0132258A0107243E142D
:0E1F50008A158619AD2F8A15A82F8A158A28A2
:02400E00023F6F
:104200006300000063000000630000006300000022
:104210006300000063000000630000006300000012
:104220006300000063000000630000006300000002
:1042300063000000630000006300000063000000F2
:1042400063000000630000006300000063000000E2
:1042500063000000630000006300000063000000D2
:1042600063000000630000006300000063000000C2
:1042700063000000630000006300000063000000B2
:1042800063000000630000006300000063000000A2
:104290006300000063000000630000006300000092
:1042A0006300000063000000630000006300000082
:1042B0006300000063000000630000006300000072
:1042C0006300000063000000630000006300000062
:1042D0006300000063000000630000006300000052
:1042E0006300000063000000630000006300000042
:1042F0006300000063000000630000006300000032
:104300006300000063000000630000006300000021
:104310006300000063000000630000006300000011
:104320006300000063000000630000006300000001
:1043300063000000630000006300000063000000F1
:1043400063000000630000006300000063000000E1
:1043500063000000630000006300000063000000D1
:1043600063000000630000006300000063000000C1
:1043700063000000630000006300000063000000B1
:1043800063000000630000006300000063000000A1
:104390006300000063000000630000006300000091
:1043A0006300000063000000630000006300000081
:1043B0006300000063000000630000006300000071
:1043C000FF00FF00FF00FF00FF00FF00FF00FF00F5
:1043D000FF00FF00FF00FF00FF00FF00FF00FF00E5
:1043E000FF00FF00FF00FF00FF00FF00FF00FF00D5
:1043F000FF00FF0001000000A0000000C800000056
:00000001FF
